:030000000211FCEE
:03000B000200C12F
:03002B000203EBE2
:03005B0002053D5E
:0300730002053350
:1000800002030406080C10182030406080020304AC
:1000900006080C101820304080FF0406080C1018C9
:1000A0002030406080A0C000000001010003020277
:1000B000010D0D040506020D0505050D06040502DA
:1000C00002C2AFC0D0C0E0205A0D302F02E473301E
:1000D000600280F90203D7306306C283C294C295DE
:1000E00085258AC25AE525F4700221CA056130606F
:1000F00013206A19758B00D0E0D0D0C283C294C29D
:1001000095D2AF32C283C294C2950201BAD26EC2F6
:100110006FE565601CC3E5611495654014C26ED23D
:100120006FC3E561956450030201BA756100020175
:10013000BA206C14C283C294C2957408D5E0FDD273
:1001400080D282D2970201BAD26FC283C294C29582
:10015000E53D20E23420E1127408D5E0FD2075026F
:10016000D297307502D2800201BA20E0127408D50D
:10017000E0FD207502D297307502D2800201BA7478
:1001800008D5E0FDD2820201BA20E11F20E00A7406
:1001900008D5E0FDD2820201BA7408D5E0FD2075D1
:1001A00002D280307502D2970201BA7408D5E0FD00
:1001B000207502D280307502D297758B00D0E0D0C6
:1001C000D0C283C294C295D2AF32D0E0D0D0D2AFE9
:1001D0003261D7E525600A207502D283307502D2DC
:1001E00095C29461D7E5256002D294207502C2952C
:1001F000307502C28361D7E525600A207502D29569
:10020000307502D283207502C283307502C29561B7
:10021000D7207502C280307502C297E525600A209A
:100220007502D283307502D295207502C29730755F
:1002300002C280C29461D7207502C280307502C2AA
:1002400097207502C297307502C2807406D5E0FD12
:10025000E525600A207502D283307502D295C294DA
:1002600061D7207502C280307502C297E525600A09
:10027000207502D283307502D295C282C29461D7B2
:10028000207502C280307502C297C2827406D5E022
:10029000FDE525600A207502D283307502D295C231
:1002A0009461D7C282E5256002D294207502C28093
:1002B000307502C297207502C295307502C2836103
:1002C000D7C282207502C280307502C2977406D5EB
:1002D000E0FDE5256002D294207502C295307502DA
:1002E000C28361D7C282E5256002D294207502C222
:1002F00097307502C280207502C295307502C283A4
:1003000061D7C282207502C297307502C28074061E
:10031000D5E0FDE5256002D294207502C2953075C6
:1003200002C28361D7207502C297307502C280E590
:1003300025600A207502D295307502D283C28220D0
:100340007502C283307502C29561D7207502C297CB
:10035000307502C280C2827406D5E0FDE525600AD0
:10036000207502D295307502D283207502C2833087
:100370007502C29561D7207502C297307502C2809E
:10038000E525600A207502D295307502D28320756A
:1003900002C280307502C297207502C28330750296
:1003A000C29561D7207502C297307502C280207550
:1003B00002C280307502C2977406D5E0FDE5256063
:1003C0000A207502D295307502D283207502C2834D
:1003D000307502C29561D7E525F4F58A758B0075F5
:1003E0006000D25AD0E0D0D0D2AF32C2AFC0D0C0BD
:1003F000E0D2D3C2CEE528600A741F552E6049159D
:1004000028814878007900E580307601F430E502F3
:1004100078FF53DACF20760343DA2030760343DACD
:1004200010C2D8C269E580307601F430E50279FF68
:10043000C3E89970CE305903752818741F552E6083
:10044000037528188858D268E52960041529815B4E
:10045000741F552E600543DA01C2D820680281ED71
:10046000E558F8C268741F552E60367982B704319A
:0F047000C3E894F0400374F0F8E8C4540F28F880
:10047F007984B7030281A1C313C313872120080214
:10048F00C313200A06C3C898F881A128F850037433
:10049F00FFF8C3E8955F5003E55FF8E52C5406704D
:1004AF003D882230630AC3E522955C4003855C22B8
:1004BF007882B60429C3E5229524401278A096408D
:1004CF000DE52426F52450097524FF0204E085224A
:1004DF0024852425C3E524955C4003855C2520CF26
:1004EF0009D0E0D0D0C2D3D2AF32C2CF7801E52845
:1004FF006008741F552E70021528C3E558940140EB
:10050F0005755B00A11CE55B046002055BE55DC33F
:10051F00240A5005755DFFA12AF55DD0E0D0D0C249
:10052F00D3D2AF32C2AF53917FC258D2AF32C2AF24
:10053F00C0D0C0E0C0F0D2D3A8FBA9FCC2D83069AC
:10054F0002A1A053DACF20760343DA1030760343AB
:10055F00DA20D269E580307601F420E502A17488B3
:10056F00268927E14053DACF20760343DA2030760D
:10057F000343DA10C2D8C269741F552E7002E126E8
:10058F007800E580307601F430E502E1268858E105
:10059F002653DACF20760343DA2030760343DA107E
:1005AF00C269205902C15A53DACF20760343DA10B9
:1005BF0030760343DA20C2D8D26988538954C3E80E
:1005CF009551F8E99552F9E4FB7AFAC3E894C8E932
:1005DF0094005008E4D2E4FB7A0AC12DC3E8946872
:1005EF00E994015008E4D2E3FB7A0FC12DC3E894DC
:1005FF00D0E994025008E4D2E2FB7A1EC12DC3E881
:10060F0094A0E994055008E4D2E1FB7A3CC12DC3D4
:10061F00E89498E994085006E4D2E0FB7A78C3E8AE
:10062F009555FCE99556FD30E708ECF42401FCEDF7
:10063F00F4FD7557007008C3EC9A50037557018885
:10064F00558956A853A95488518952C3E89526F85D
:10065F00E99527F9307402C1F9307302C1F930728C
:10066F0002C1F2E9C313F9E813F8307102C1F2E9DC
:10067F00C313F9E813F8307002C1F2E9C313FDE8B0
:10068F0013FC205918C3EC941CED9402400302078D
:10069F0026ED7009C3EC94C8500302074074002084
:1006AF0077037896E624FAFEE43400FFC3EC9EFC51
:1006BF00ED9FFD500678007900C1F9C3EC94FFED72
:1006CF009400400678FF7900C1F9EC856CF0A4C561
:1006DF00F0A2F733F87900400302071578FF79008D
:1006EF00020715E9C313F9E813F830740EE9600235
:1006FF0078FFC3E81338F8E43400F9C3E894FFE94E
:10070F009400400278FF8858D268205902E126747D
:10071F001FF4552E4BF52E752818741F552E700388
:10072F0075280A305902E140741F552E600353DAC1
:10073F00FE752906741F552E700375290AD0F0D047
:10074F00E0D0D0C2D3D2AF327901E16F7903E16F3C
:10075F00790AE16F791EE16F7964E16F79C8E16F12
:10076F007817E4D5E0FDD8FAD9F6227A147B78020F
:10077F0007967A107B8C0207967A0D7BB402079648
:10078F007A0B7BC8020796AC257525017902B275E5
:10079F00E4C282D5E0FDE5256002D294D5E0FDC22A
:1007AF0094D5E0FDD282D5E0FDE525600A207502E3
:1007BF00D283307502D295E56DD5E0FD207502C26A
:1007CF0083307502C2957496D5E0FDD9C1EAF8D58C
:1007DF00E0FDD8FBDBB1C2828C2522C37C007D00FB
:1007EF0075F00005F0EA33FAEB33FB50F6EB13FB31
:1007FF00EA13FAC3E9FFE8FEE89AF8E99BF9500417
:10080F00EFF9EEF8B3EC33FCED33FDD5F0DFEDF996
:10081F00ECF822E889F08A20D2D4F8A9F07B0030D6
:10082F00F70B7BFFF42401F8E9F43400F9E8852095
:10083F00F0A4ADF0F8E98520F0A4AFF0FEED2EF9AD
:10084F0074003FFA7C04C3EA13FAE913F9E813F8CA
:10085F00DCF48BF030F70AE8F42401F8E9F4340003
:0F086F00F9E889F0C2D4F8A9F0227882B6040320
:10087E000208D6C3E5589401400302089E8522243F
:10088E00E4F53FF540F541F542F543F5480208D64B
:10089E007882E6FC754801E522F523783879C7AAF7
:1008AE003BAB3CC3EB13FBEA13FAEC146013C3EB44
:1008BE0013FBEA13FAEC14146007C3EB13FBEA13F1
:1008CE00FA1207EA883F894022E5486034C3E53FC3
:1008DE009523F8E5409400F9500CC3E89480E99410
:1008EE00FF401602090BC3E8947FE99400500302FF
:1008FE00090B787F790002090B788079FF8844898B
:10090E004522E5486058E5442541F8E5453542F96C
:10091E00854520E4300701F43543FA30E709C3EA90
:10092E0094F0401502094DC3EA940F500302094D8D
:10093E0078FF79FF7A0F02094D780079007AF0C3BB
:10094E00E524955C5006E52460092166E54520E71F
:10095E000D2166E54530E706884189428A4322E546
:10096E004870030209D0789EE6FAC3E54433F8E5F1
:10097E004533F91122E930E70BC3E89480E994FF7F
:10098E00401321A7C3E8947FE99400500221A77871
:10099E007F790021A7788079FFE820E715C3E5234A
:1009AE0098F84009C3E8940140030209CE78010289
:1009BE0009CEE8F424012523F840030209CE78FF7E
:1009CE00884622E5487003020A32789FE6FAA8426A
:1009DE00A9431122E930E70CC3E89401E994FF40E2
:1009EE0016020A09C3E894FFE994005003020A09AB
:1009FE0078FF7900020A09780179FFE920E715C32B
:100A0E00E54698F84009C3E894014003020A30789D
:100A1E0000020A30E8F424012546F84003020A30A9
:100A2E0078FF8824227883E6F520120F7075E890FF
:100A3E00E5E820ECF0A8BDA9BE1210057568557545
:100A4E006900C3740013FD745513FC74552CFC74AB
:100A5E00003DFDECFAEDFBC3E89AE99B4014E56816
:100A6E002455F568E5693400F569EA2CFAEB3DFB8F
:100A7E0080E5AE68AF69C3E56913F9E56813F8C39D
:100A8E00E913F9E813F8E56828F566E56939F567BD
:100A9E007A03C3E913F9E813F8DAF7AA201A7009F2
:100AAE00756800756900020AC71AEA6008EE28FE2A
:100ABE00EF39FFDAF88E688F692275E89022788315
:100ACE00E6FFE5E820ECF7A8BDA9BE056AC3E56A16
:100ADE0094084052756A00E97007E56B601B020AC4
:100AEE00FBC3E8956B6010E56B5006600C14020BAF
:100AFE00070460F9020B07E56BF56BC3946DF840C4
:100B0E0021755CC0C3E89404F84017755C80C3E897
:100B1E009404F8400D755C40C3E89404F8400375E6
:100B2E005C0075BB0922EFC39401601BC3E894FF00
:100B3E00E994035012C3E89568E995695009E55C9C
:100B4E00600C155C020B5CE55CF46002055CA85C55
:100B5E00C3E524985002A8248825C3E525955D4059
:100B6E000B855D25E55DF46003855D5CC3E56AB4C8
:100B7E00070375BB1022306102783230620278783A
:100B8E00E52C5406601FE879A187F0A4C5F0A2F702
:100B9E0033F8C3E8955C4002A85C88228824882537
:100BAE00306102885E22788FE6FFC3EF94055018FD
:100BBE00C3EF94045020C3EF94035028C3EF940264
:100BCE005030C3EF940150387533A075340F75351E
:100BDE003C753605811C7533C075341275354075FC
:100BEE003606811C7533707534177535D07536071A
:100BFE00811C75334C75341D7535C4753609811CD1
:100C0E007533287534237535B875360B811C8533CD
:100C1E004F853450753B00753C0822A84FA95002F1
:100C2E000C34A849A94A759100C3E498F594E49947
:100C3E00F595759104D25875C820A8CCA9CD75C864
:100C4E0024AA39AB3A8839893AC3E89AF8E99BF96C
:100C5E00AA3BAB3CC3EB13FDEA13FCC3ED13FDEC57
:0F0C6E0013FCC3EA9CFAEB9DFBEA28FAEB39FB77
:100C7D008A3B8B3C400122753BFF753CFF2230586F
:100C8D0002818B759100C3E4954BF594E4954CF579
:100C9D0095759104D258227892E6FF7E10305B0252
:100CAD007F053063047F037E00A93CA83B7A04C313
:100CBD00E913F9E813F8DAF7C3E89EF8E99400F9B7
:100CCD004009C3E89402E9940050047802E4F9E97C
:100CDD00FBE8FAC3E913FDE813FCC3EF9403602EA0
:100CED00EF20E00DE82CF8E93DF9ECFAEDFB020DF3
:100CFD0008E828F8E939F97A02E4FBC3EF940340D8
:100D0D000D8A4D8B4E8849894A8C4B8D4C22884DCE
:100D1D00894E8A498B4A8C4B8D4C22305802A12822
:100D2D00759100C3E4953BF594E4953CF59575916B
:100D3D0004D25822753E00752000020D50753E00FC
:100D4D00752040D2AF053E20580122759D00E53C2F
:100D5D00C313C313F8086030306A06C313C313F806
:100D6D0008C3E8940A4002780A306D08C3E8940479
:100D7D0040027804C3E53C9408400D759D02C3E51F
:100D8D003C94104003759D03205803D2AF22791E69
:100D9D00206D02790AD2AF0000C2AF205A0A793C09
:100DAD00206D027914306FE03063027978C3E58BE2
:100DBD009920630240F740D0E59BF4F45440B520F0
:100DCD0002A150D8C3D2AF22C25B789CE614600753
:100DDD00E53E147002D25B30630B05382058107558
:100DED003800020DFC205807158115810217452288
:100DFD00759100C3E4954DF594E4954EF595759177
:100E0D0004D25822AE25305B4F78A3E6FFBF010B0D
:100E1D00D25C752500C283C294C2959190305C035B
:100E2D00752500305802C12ABF020BD25C75250012
:100E3D00C283C294C29578A2B6010D9190305C0325
:100E4D00752500305802C14ABF030BD25C752500D1
:100E5D00C283C294C295B1FD305C03752500305834
:100E6D0002C165305B04C25C8E2522C2AFC28220F6
:100E7D006A03020E9790034B306E0F207502C297D6
:100E8D00307502C2807406D5E0FD207502D2803027
:100E9D007502D297759F43753D02D2AF22C2AF2026
:100EAD006A03020ECC900302306E17C282207502C7
:100EBD00C297307502C2807406D5E0FD020ECF9048
:100ECD0001E5207502C295307502C283305A06E5E0
:100EDD00256002D294207503759F53307503759F5D
:100EED0033753D03D2AF22C2AF207502C28030757B
:100EFD0002C297206A03020F139002C1306E07C21F
:100F0D00827406D5E0FD207502D297307502D2802D
:100F1D00207503759F33307503759F53753D04D24E
:100F2D00AF22C2AF206A03020F51900280306E17BC
:100F3D00207502C280307502C297C2827406D5E058
:100F4D00FD020F549001D3C294305A0EE525600A6C
:100F5D00207502D283307502D295759F43753D057C
:100F6D00D2AF22C2AF207502C297307502C2802067
:100F7D006A03020F97900237306E0F207502C28000
:100F8D00307502C2977406D5E0FDD28220750375C7
:100F9D009F53307503759F33753D06D2AF22C2AF97
:100FAD00206A03020FD59003A4306E1F207502C274
:100FBD0080307502C297207502C297307502C280CB
:100FCD007406D5E0FD020FD89001F7207502C2839B
:100FDD00307502C295305A0EE525600A207502D291
:100FED0095307502D283207503759F333075037567
:100FFD009F53753D01D2AF229001D1C283C294C2DD
:10100D0095C280C282C29722C3E54F9535E55095B2
:10101D00365001227890E6FFC3EF94055018C3EFC8
:10102D009404501BC3EF9403501EC3EF9402502140
:10103D00C3EF94015024C3E54F943CF8021070C3E4
:10104D00E54F9428F8021070C3E54F941AF802107A
:10105D0070C3E54F9412F8021070C3E54F940AF86F
:0D106D00021070E5509400F9884F89502260
:10107A0030580302107A22788076077881760778CA
:10108A008276017884760378837601788676097881
:10109A008F7601789076057895760278927603783D
:1010AA009B760D7893760678877601789C76027817
:1010BA008876017889760178857600788C76017849
:1010CA008D7600788E76B478967625789776D0786D
:1010DA00987678789976C8789A7604789D760022F8
:1010EA007893E6FF756409756501C3BF02097564E3
:1010FA000575650102112FC3BF030975640575657E
:10110A000202112FC3BF0409756405756503021134
:10111A002FC3BF0506756409756507C3BF06067543
:10112A0064007565007887E6FFC26CC3BF0302D20C
:10113A006CC26BC3BF0402D26BC26A7418552D60AD
:10114A0002D26AC26E6002D26ED26F6002C26FC2EF
:10115A00757888E630E102D275C2767889E630E1A0
:10116A0002D276C3EF94026008758E01D26D021125
:10117A0080758E00C26D227880E614900080937884
:10118A009EF67881E61490008093789FF6110522E6
:10119A00789BE61490008D9378A0F6110522788644
:1011AA00E61490009A9378A1F6110522789CE61429
:1011BA009000A79378A2F6789CE6149000AC9378F6
:1011CA00A3F6110522227896E6FA7897E6FB30779D
:1011DA00047A007BFFC3EB9AFCC3948250027C82A0
:1011EA00756C00056CEC856CF0A4C3E5F094804046
:1011FA00F222C2D353D9BF7581C043FF8012075769
:10120A0075EF0243B203E5B324044002F5B37580D7
:10121A00F275A40D75F13F75D4DF75904F75A5B0C1
:10122A0075F2F075D50075A60175E2411105E4F86D
:10123A00F6D8FD118112177311EA3181319A31A85A
:10124A0031B631CF31D07898866D110575885075D1
:10125A00890275C82475910475D84012076B120764
:10126A007A1207631207811207631207881207634B
:10127A00121CE512076B12076B12076775A8227515
:10128A00B80275E69075F610759B80759D0375D149
:10129A000E75BC5875BB0975BA1175E880120757E7
:1012AA00D2AF120A3343DA01C2D8C26912076B7588
:1012BA003001D2597A05E55770027A0512075BE5C3
:1012CA0058C3940240EEE52E541F855A59F55AB573
:1012DA0059E2DAE2C25953DACF20760343DA2030F0
:1012EA00760343DA10C2D8C26912076712075B781D
:1012FA0002741F552E70027800C3E5589840EDC25B
:10130A00AF12077A12077A12077AD2AF12076B75F1
:10131A00470012075B788CE6C3940150030213E579
:10132A00E530C3940150030213E5741F552E60354E
:10133A00C3E55894FF50030213E5C2AF12078FD2D8
:10134A00AF120767C3E558940150EFC2AF12077A8C
:10135A0012075F12077AD2AF120767C3E55894FFE4
:10136A0040E9021D6A7F05D27731D0120767C2AF02
:10137A00C27731D0C3E558947FD2AF4068C2AF126A
:10138A00078FD2AFDFE1C3E55894057897F61207C5
:10139A006B121822121CED7F0AD27731D01207671E
:1013AA00C2AFC27731D0C3E558947FD2AF50E8C2FA
:1013BA00AF12077A12075F12077AD2AFDFDBE5585E
:1013CA0024057896F612076B121822121D1C1207B2
:1013DA0067C3E55894FF40F6021D6AC3E55895476E
:1013EA004003855847120767C3E5589401400261D4
:1013FA001CC2AF12078F12078F12078FD2AF1207C4
:10140A006B753000E4F531F5320531E531F47036AB
:10141A000532789AE67828146012785014600D78AC
:10142A00A014600878F0146003753200C3E532989E
:10143A00401415327899866DC2AF12078FD2AF78F1
:10144A0098866D12076712075BE5287008741F55A6
:10145A002E700241BCC3E558940640AD120767E5F9
:0F146A002870030212BC1105E4F522F523F524C6
:10147900F525755CFF7885865FF53FF540F541F503
:1014890042F543F56AF548F52BF52CF55B120BB4DB
:10149900756A0875BB10120757120AC8E5E820ECEF
:1014A900FBA8BDA9BEE97001F8886B120ACC756A60
:1014B9000875BB107895E630E0030215027887E6D7
:1014C900FE760211EA7887EEF6D261C2AF120B847A
:1014D90085225C85225DD2AFC261752500756200E7
:1014E900756301D260D263753800120F70120FABA9
:1014F900120C30120BB402162B7887E6FE760378AD
:1015090093E6FD760511EA7887EEF67893EDF6D243
:1015190060D261D26E120F70120FAB120B841207D8
:1015290057120E78120757120757120EAA12075BA5
:10153900120EF412075B12075B120F2F12075F12CC
:101549000F7012075B120757C261D262120AC812E2
:101559000ACC120B84756A0875BB10120FAB120CFA
:1015690029120CA41115117A120E78120C29120CD9
:10157900A41115117A120EAA120C29120CA4111514
:10158900117A120EF4120C29120CA41115117A12E7
:101599000F2F120C29120CA41115117A120F7012A7
:1015A9000C29120CA41115C3E54F9535E550953654
:1015B900400C117AC3E55894015091021745117AEC
:1015C900C2627887E6FE760211EA7887EEF685220E
:1015D9005C855E5D855E25756200756301D2637504
:1015E9003800C2AF207502C280307502C2972075DB
:1015F90002C297307502C280742DD5E0FDD2AF12B8
:101609000FAB120C30120C8B120CA4120D28756A38
:101619000075BB0902162B11EA120FAB756A00752A
:10162900BB09120D4A120DD5120DFD120879120EC1
:1016390011120E78120C30120C8B120CA4120D28F8
:10164900120D41120DD5120DFD1208D7120E1112ED
:101659000EAA120C30120C8B120CA4120D28120DAA
:101669004A120DD5120DFD120910120E11120EF4A7
:10167900120C30120C8B120CA4120D28120D4112EF
:101689000DD5120DFD12096D120E11120F2F120C2C
:1016990030120C8B120CA4120D28120D4A120DD502
:1016A900120DFD1209D1120E11120F70120C301207
:1016B9000C8B120CA4120D28120D41120AC8120D1E
:1016C900D5120DFD120ACC120E11120FAB120C30ED
:1016D900120C8B120CA4120D2830632A855E5C85CE
:1016E9005E5D756200756301C3E5389464400AC2A2
:1016F90063D26475371402170FC3E5589401400388
:1017090002162B021745306419E537147005C264B7
:10171900021620F537C3E5589401400302162B023F
:101729001745C3E55B94FA5013741F552E7004E5F1
:10173900286009C3E53C94F05002C12B1105788754
:10174900E6FE760211EA7887EEF6E4F522F523F54E
:1017590024F525F55FC2601207571105741F552E30
:101769007006E528700241BC810E901A0D7820128E
:101779001C00E520B4550CA3121C00E520B4AA03F3
:101789000217941181121822021821901A037880E5
:10179900121C00A308121C00A308121C00901A06B0
:1017A9007883121C00A308121C00A308A308121CAA
:1017B90000A308121C00A308121C00A308121C0095
:1017C900A308A308A308121C00A308A308121C005D
:1017D900A308121C00A308121C00A308A308121CCA
:1017E90000A308121C00A308A308121C00A30812D6
:1017F9001C00A308121C00A308121C00A308121C39
:1018090000A308121C00A308121C00A308121C0044
:10181900A308121C00901A2122C2AF121C3F121CED
:1018290019901A00740A121C05A37404121C05A34A
:101839007410121C05901A037880121C04A3081254
:101849001C04A308121C04901A067883121C04A312
:1018590008121C04A308A308121C04A308121C04E0
:0F186900A308121C04A308121C04A308A308A3BD
:1018780008121C04A308A308121C04A308121C04C1
:10188800A308121C04A308A308121C04A308121C12
:1018980004A308A308121C04A308121C04A308121A
:1018A8001C04A308121C04A308121C04A308121C7D
:1018B80004A308121C04A308121C04A308121C0485
:0A18C800121C52121C30901A21224B
:101A00000A04100909040103FF0901010155AA0193
:101A1000FFFF0105FF0306FF0225D02850040D0239
:021A200000FFC5
:101A400023416C69676E424C333558232020202097
:101A500023424C48454C4923463333302320202031
:101A60002020202020202020202020202020202076
:101C0000E493F622E6438F01538FFD75EF0275B71B
:101C1000A575B7F1F0538FFE22438F02438F0175F4
:101C2000EF0275B7A575B7F1901A0DF0538FFC222E
:101C3000901A0D74559105901A0E74AA9105227A86
:101C40003079D07820901A409100E520F709A3DA86
:101C5000F7227A3079D0901A40E7910509A3DAF992
:101C600022AB6EA86FBB01057980021CE2BB0205A6
:101C70007981021CE2BB03057982021CE2BB0405E8
:101C80007984021CE2BB05057983021CE2BB0605D0
:101C90007995021CE2BB07057986021CE2BB0805A8
:101CA000798F021CE2BB09057990021CE2BB0A0590
:101CB0007992021CE2BB0B05799B021CE2BB0C056E
:101CC0007993021CE2BB0D057987021CE2BB0E056D
:101CD000799C021CE2BB0F057988021CE27989021B
:101CE0001CE2E8F7227C0512076BDCFB22C2AF1274
:101CF000077A12078112078812078F12075F1207EF
:101D00007A12078112078812078F12075F12077A6B
:101D100012078112078812078FD2AF22C2AF1207B3
:101D20008F12078812078112077A12075F12078F36
:101D300012078812078112077A12075F12078F12A3
:101D4000078812078112077AD2AF22AE6EAF6FC238
:101D5000AF12077A12077A12077A12075FDEF212C1
:101D6000078F12075FDFF8D2AF2291ED91E591E581
:101D7000756E01756F01757000B14B7C05AD581221
:101D8000076BC3ED955870F5C3E55894014009C33E
:101D9000E55894FF4032A1A6916112182291EDC23C
:101DA000AF75EF1291E5DCD50570C3E57094035073
:101DB0000280C691E5056FE56E149000B193F808B6
:101DC000C3E56F98500280AE91E591E5056EC3E5DD
:101DD0006E94115002809C121081121822C2AF75AD
:041DE000EF1291E588
:00000001FF
